:020000040800F2
:10000000C8080020C9000008612900080124000870
:1000100000000000000000000000000000000000E0
:10002000000000000000000000000000652900083A
:100030000000000000000000632900086729000894
:10004000DB00000800000000DB000008DB00000807
:10005000DB000008DB0000086905000873050008E4
:10006000000000003905000849050008590500088E
:1000700055020008DB000008DB000008000000005B
:10008000DB00000800000000000000005D2A0008FE
:1000900000000000DB000008DB000008DB000008B7
:1000A00000000000DB0000080000000049320008EA
:1000B0000448854600F0BCF800480047B533000806
:1000C000C046C046C808002004488047044800478E
:1000D000FEE7FEE7FEE7FEE7FEE7FEE75B2A000835
:1000E000B100000830B50B46014600202022012453
:1000F00009E00D46D5409D4205D31D469540491B5C
:100100002546954040191546521E002DF1DC30BDA4
:1001100070B500242546002801DA01244042002958
:1001200001DA01254942FFF7DDFFAC4200D0404231
:10013000002C00D0494270BDF0B51FB40646002027
:1001400082B005464024019100901BE001992246AF
:100150000F46304600F020F8049A059B801A99411A
:1001600010D310461946224600F052F8361A8F4135
:100170000197224601200021009F00F049F838181D
:100180004D4100902046641E0028DFDC019B009852
:100190002946324607B0F0BD10B5202A04DB0846D8
:1001A000203AD040002110BD0B46D340D04020243F
:1001B000A21A91400843194610BD03460B439B0702
:1001C00003D009E008C9121F08C0042AFAD203E0CC
:1001D0000B780370401C491C521EF9D27047D2B2F2
:1001E00001E00270401C491EFBD270470022F6E776
:1001F00010B513460A4604461946FFF7F0FF20469D
:1002000010BD421C0178401C0029FBD1801A7047A8
:1002100010B5202A04DB0146203A9140002010BD91
:10022000914020239C1A0346E3401943904010BD9F
:10023000064C0125064E05E0E36807CC2B430C3C39
:1002400098471034B442F7D3FFF736FFCC37000895
:10025000EC37000810B5024800F05BFA10BD000052
:10026000BC02002070B5044600688168490727D5A4
:10027000816810254907002905DA8168890702D4B9
:1002800081682943816000F065FF06462068806828
:10029000400715D500F05EFF801B02280CD92068AE
:1002A0008068400708D5A06B2843A063E06B01215C
:1002B0000843E063084670BD206880684007E9D4C1
:1002C000002070BD10B50246406A816B5023194270
:1002D0000AD1816B01225202114381630168CA680D
:1002E0001205920F05D020E0006B016B1046884785
:1002F00010BD827E002A18D10A68120715D58A68B7
:1003000001235207002A09DB4A680C24A2434A60F1
:10031000816B1A0291431943816306E0816B2022AD
:1003200011438163C16B1943C16300F0EFF910BD44
:1003300010B5406A816B402211438163C16B042276
:100340001143C16300F0E4F910BD10B5406A00F03C
:10035000DEF910BDF8B50446006881688907890F89
:1003600001292FD10168C90702D1C168090429D523
:1003700081680522114010250126012916D18168C6
:1003800002221143816021680320086000F0E2FE30
:10039000074620688068C00714D000F0DBFEC01B51
:1003A00002280BD920688068C00707D0A06B2843BB
:1003B000A063E06B3043E0630120F8BD20688068F3
:1003C000C007EAD10020F8BDF8B50446002000902F
:1003D000206881688907890F012905D10168C9074B
:1003E00036D1C168090433D481681A4A10261140F5
:1003F000012500291FD181682943816017481649CA
:100400000068FFF76FFE0090002802D0401E0090A9
:10041000FCD100F09FFE074620680068C043C0077B
:1004200016D000F097FEC01B02280CD92068006887
:10043000C043C00707D0A06B3043A063E06B2843E4
:10044000E0630120F8BD20680068C043C007E8D120
:100450000020F8BD1700008040420F00340000204B
:1004600010B5204C012023881A464100615A994258
:1004700001D90B4602E0914200D20A46401CC0B2AC
:10048000FA28F2D3981A184C002802DDE1894018A6
:10049000E0812079411C2171042822D30E200521FE
:1004A000205EFFF735FE114948431149FFF730FE42
:1004B0001621615E00B248430A21FFF729FE01219F
:1004C0006156414308B2E081A081E178012902D060
:1004D000002902D002E0208200E060820020E0815A
:1004E000207110BD3800002000000020E40C000046
:1004F000FF0F0000417802780802104340BA7047AD
:1005000070B4FF234A1E1C4692B200290CD0084D3D
:10051000084E0178401C59406B5C6340745C114686
:10052000521E92B20029F4D11802204370BC7047C9
:10053000B4350008B436000810B5024800F03AFBA4
:1005400010BD0000FC02002010B5024800F032FB94
:1005500010BD00001C04002010B5024800F02AFB6A
:1005600010BD00006004002010B5082000F024FD3C
:1005700010BD10B5802000F01FFD10BD72B6FEE763
:1005800070B5044600F0E6FD1A4D0646E868C0075F
:100590000DD0601C08D0002C04D000F0DBFD801BC7
:1005A000A04201D9032070BDE868C007F1D1E86816
:1005B000800601D52020E860E868C00602D4E8681B
:1005C000400715D5E9680020CA060B4904D5C8695B
:1005D00002221043C8611020EA68520705D5CA6993
:1005E00001231A43CA6104210843E860012070BD59
:1005F000002070BD00200240A8040020F8B50025AE
:10060000044620340095227D012A39D00126267522
:10061000026893685B0767D4384F4B68BB424DD084
:10062000936A0F78BE40334393620123C26A1B076B
:100630009A421FD0012A1DD0022A1BD0032A19D0AA
:10064000042A17D0052A15D0062A13D0072A11D05C
:1006500002688B6856697607760FB3420AD05369F1
:10066000DB08DB005361006842690B7A5B075B0FB4
:100670001A4342610868102804D0112802D038E0DB
:100680000220F8BD1E4B9A68102807D00120800573
:1006900002439A600868102803D02AE00120C005B0
:1006A000F6E7194817490068FFF71CFD0A2148437F
:1006B00000901ED0401E0090FCD11AE0906A0B788A
:1006C0009E40B04390620868102801D0112810D1D4
:1006D0000B498A68102804D00120800582438A6073
:1006E00007E00120C005F9E7816B202211438163F7
:1006F0000125002020752846F8BD000001100000EB
:100700000027014040420F0034000020704770472E
:10071000704770B5044600680168490702D5416812
:10072000490705D40168090730D5416809072DD567
:10073000A16BC90604D4A16B012252021143A1632B
:10074000C1680C250905890F00291AD1A17E00294D
:1007500017D10168090714D58168012249070029CA
:1007600008DB4168A9434160A06B11028843104334
:10077000A06306E0A06B20210843A063E06B104358
:10078000E0632046FFF7C2FF20680560206801682B
:1007900009060DD5406800060AD5A06B01210904A1
:1007A0000843A063204600F0D9F821688020086043
:1007B00020680168C90613D54168C90610D5A16A29
:1007C0001025012902D0C168C90707D0E16B0222B8
:1007D0001143E16305602046FFF79AFF206805603A
:1007E00070BD0000F8B500250446002805D0A06BB8
:1007F00026462036002802D007E00120F8BD002060
:10080000E0633075204600F0ABF8A06B1022C00604
:10081000002870DB2068816849076CD4A16B130144
:10082000994302231943A16381688907890F01292C
:1008300005D10168C9070FD1C16809040CD4C1688A
:1008400018239943A3681943C1602068016963684C
:1008500089008908194301612068C1683D4B19402E
:10086000C160207E8103607EC0030143A07E4303FC
:100870001943A36A012B02D001231B0300E00023CC
:100880001943E36819432369022B09D00023194354
:100890003379E67E5B0019430123012E02D00AE082
:1008A0000423F4E7002827D0A06B20263043A06360
:1008B000E06B1843E063E0690646FF3EC23E02D0AB
:1008C000266A304301432068C6680E43C66001268D
:1008D000E06A3607B04213D0012811D002280FD0A9
:1008E00003280DD004280BD0052809D0062807D0EE
:1008F000072805D010E028E0012000040143DAE7D2
:1009000020684669F608F600466120684669A78DAA
:100910007F077F0F3E4346612068C0680E4E30401F
:10092000884207D10020E063A06B80088000401C53
:10093000A06308E0A06B022188431043A063E06B32
:100940001843E06301252846F8BDA06B1043A0635F
:10095000F8E700001902FEFFE7FF3F837047000041
:1009600070B586B000240546009401940294039467
:10097000049400681E49884237D11E488169421597
:100980001143816181691140059142690121490446
:100990000A4342614069084005900220009003200C
:1009A000019009206946C00600F012FB134E124860
:1009B0007460B46030608020F0604000306180007E
:1009C00070612020F461B061304600F045F90028E4
:1009D00001D0FFF7D3FD2E63002211460C20756273
:1009E00000F052FC0C2000F043FC06B070BD00008B
:1009F000002401400010024008000240FC020020D8
:100A0000F7B5044600680025806840073ED42646B6
:100A10002036307D01280AD001273775607E0128F5
:100A200008D02046FFF7D0FC050003D02FE00220BD
:100A300003B0F0BDA06B17490840FF210131084306
:100A4000A0630020E0633075216B13488862216B3E
:100A50001248C862216B1248086321681C20086094
:100A6000206841681022114341602068C168394301
:100A7000C1602168206B4031029B019A00F020F98F
:100A80002068816804221143816000E00225284625
:100A900003B0F0BDFEF1FFFFC50200084B030008E4
:100AA00031030008F8B5064604462036307D01289B
:100AB00007D0012737752046FFF7D4FB050002D089
:100AC0002AE00220F8BD2068C16849084900C160D9
:100AD000206B014620304078022808D1084600F0FB
:100AE0001FF8050003D0A06B40210843A0632068D5
:100AF0004168102291434160002D204602D0FFF74B
:100B000029FC09E0FFF726FC050005D1A06BFF21B9
:100B1000013188433843A063002030752846F8BD72
:100B2000014620314A780023022A04D0042282633D
:100B30000B700120704730B4026814680E25AC4376
:100B40001460026814686408640014600125046C71
:100B50002A46C06BA24042604D700B7030BC002032
:100B6000704770B50024014620314A78022A03D02C
:100B700004218163012416E0026813680E25AB434B
:100B80001360026813685B085B0013600125036C47
:100B90002A469A40C36B5A604D7000220A70416B1E
:100BA000002900D08847204670BD806B70472030F8
:100BB00040787047F0B4C16B0C6801680B6804267C
:100BC000056C3246AA40224210D05A070ED50A6858
:100BD000920602D40A68B2430A60016C8E40C16B6F
:100BE0004E60C16A002935D1F0BC70470227AF4082
:100BF0000246274001262032002F15D09F0713D52B
:100C00000B689B0604D40B680A24A3430B60567040
:100C1000036C02219940C36B596000211170816AF5
:100C2000002917D1F0BC70470827AF402742F9D000
:100C30001B07F7D50B680E24A3430B60016C3346EA
:100C40008E40C16B4E608363537000211170016B45
:100C50000029E7D0F0BC0847002801D101207047E7
:100C600070B5044602202546203568702068026869
:100C70001049A3680A40616826691943E368334351
:100C8000194363691943A3691943E369194311437C
:100C900001600949206840181421FFF723FA8000F9
:100CA00020640648E0630020A06301216970287079
:100CB00070BD00000FC0FFFFF8FFFDBF0000024045
:100CC000F0B404469446203422780025012A0AD044
:100CD0000127277066780022012E07D02270022596
:100CE0002846F0BC7047F0BC0220704702266670B0
:100CF000826302681468640864001460046C3E46F1
:100D0000A640C46B62466660046863604368102B4B
:100D100003680AD099600168CA60C16A0029016845
:100D20000A6806D00E231A430AE09A600268D1606E
:100D3000F3E70A231A430A6001680A6804239A4306
:100D40000A600068016839430160C9E7F3B50546E8
:100D500081B0012000902E48017E01290DD0012193
:100D6000017628682B4C2C4E4027012808D02046BD
:100D7000FFF706FC002819D044E0022003B0F0BDC4
:100D80002046FFF7FDFB00283CD12149C8613069AE
:100D90000425284330613069384330612046FFF72D
:100DA000EFFB00903069A84330612BE000210298EE
:100DB000C9430160A8686C6880020019A04221D96B
:100DC00013490020C86130690227384330617461DB
:100DD00030694021084330610E48FFF7D1FB009095
:100DE0003069B84330610098002802D0029804604E
:100DF00008E0012080022418A86869688002401871
:100E0000A042DDD8024900200876009803B0F0BD6A
:100E1000A804002050C300000020024003480169DC
:100E20008022114301610020704700000020024031
:100E3000F0B51FB405461D480024017E012907D0E6
:100E4000012606761A48FFF79BFB002803D027E00F
:100E5000022005B0F0BD012D02D0022D00D00425E6
:100E6000002D1DD9134E019861000F18220103991E
:100E70000298FFF791F90D4A0021D16131690122F1
:100E80001143316138800A48FFF77AFB316949081C
:100E900049003161002803D1641CE4B2AC42E2D3C2
:100EA000024A0021117605B0F0BD0000A804002020
:100EB00050C3000000200240064900200A691206C3
:100EC00007D5054A4A60054A4A600969090600D5FE
:100ED000012070470020024023016745AB89EFCD18
:100EE000F8B509270025FF060126304C802815D0CB
:100EF00008282CD12E49022002F032FA0821384667
:100F000000F014F9012823D0E5701020205E294953
:100F1000421849008A423DD9962045E04021384692
:100F200000F004F9012802D1A079401CA071607979
:100F3000401CC0B26071052809D9A079032801D3EB
:100F4000667002E00020C04360706571A571F8BD55
:100F5000E67010201221205E615E228B401A032170
:100F600090420BDDE079401CC0B2E071032801D350
:100F7000A5702572FA28EAD9E171F8BD207A401CE3
:100F8000C0B22072032801D3A670E571FA28F4D903
:100F90002172F8BD7D21FF30C900F530884202D9A9
:100FA00064202083F8BD28202083F8BD00000020A5
:100FB00088130000DC05000004494A69024204D09D
:100FC00010B54861FFF78CFF10BD70470004014069
:100FD0000B680022002B72D0F8B401270B689740F1
:100FE0003B406DD00C79A407A40F012C01D0022C3A
:100FF00010D1856854000326A640B543CE68A640AC
:101000002E43866044680D79BC43ED06ED0F954094
:10101000254345600C79E443A40708D0C568540013
:101020000326A640B5438E68A6402E43C6600C79C1
:10103000A407A40F022C0CD1D408A40027183D6AE1
:101040005407E40E0F26A640B5430E69A6402E4372
:101050003E62056854000326A640B5430E79B607E4
:10106000B60FA6402E4306604C68A403A40F49D0D7
:10107000284CA56901263543A561A469950834402B
:101080000094254CAD002F19BD689407240F0F263E
:10109000A640B5430926F606B04201D1002611E06C
:1010A0001E4EB04201D101260CE01D4EB04201D1CE
:1010B000022607E01B4EB04203D1032602E028E0DF
:1010C00020E00526A6402E43BE60174D2C684E68D2
:1010D0009C43F60300D51C432C606C684E689C430F
:1010E000B60300D51C436C60AC684E689C43F602A6
:1010F00000D51C43AC60EC684E689C43B60200D53A
:101100001C43EC600B68521CD34000D065E7F8BC70
:101110007047704700100240000001400004004882
:1011200000080048000C0048000401400069084025
:1011300000D001207047426913460B401B049143C5
:101140000B4383617047002A01D08161704781623F
:1011500070470000014880687047000028000020A8
:10116000002801D10120704770B504462168164857
:10117000086021681548086020686168416021683E
:10118000A0688860FFF7E6FF05462068C068400752
:101190000ED0FFF7DFFF401B272805D92068C06865
:1011A000400701D0032070BD2068C0684007F0D11F
:1011B00020680269E1688A4201D0016101E00449C6
:1011C0000160002070BD0000CCCC0000555500002F
:1011D000AAAA0000006802490160002070470000D0
:1011E000AAAA000010B50648016810221143016048
:1011F000032000F007F800F027F8002010BD0000E1
:101200000020024070B504460D4D7D202978C000B5
:10121000FEF768FF01460B480068FEF763FF00F029
:1012200099FB002809D1042C07D200222146401E38
:1012300000F02AF800206C6070BD012070BD000035
:101240002800002034000020084881B08169012274
:1012500011438161816911400091C26901040A430F
:10126000C261C0690840009001B0704700100240A0
:10127000002805DBC106C90E01208840014908602D
:101280007047000000E100E08207D30EFF229A4081
:101290008907090E9940002808DB830809489B004C
:1012A0001818036893430B43036070470007000F4F
:1012B0000838830804489B001818C36993430B43FC
:1012C000C361704700E400E000ED00E0F8B50446BB
:1012D0000068394EC0035AD5F0690025C00007D414
:1012E000F06931040843F061F0690840012500907D
:1012F00032480168C90515D40068FF21013108434F
:101300002E490860FFF726FF07462C480068C005F5
:1013100008D4FFF71FFFC01B642825D827480068A2
:10132000C005F6D5306A03210902084021D0626861
:101330000A4082421DD0306A326A88430121090482
:101340000A433262326A8A4332623062C00710D086
:10135000FFF700FF0746306A80070AD4FFF7FAFE5E
:10136000C11B1748814201D90320F8BD306A8007AC
:10137000F4D5306A0321090288436168084330626A
:10138000002D04D0F069012109078843F06120781D
:10139000C00705D0306BA168800880000843306327
:1013A0002078800605D5306B10218843E16808431A
:1013B00030630020F8BD00000010024000700040C3
:1013C00088130000002801D101207047F8B50446B9
:1013D0003E480D460068C007C00FA8420AD23B48ED
:1013E000016849084900294301600068C007C00F2F
:1013F000A84250D12068364E81070CD5400704D54D
:10140000706807210902084370607068F021884302
:10141000A168084370602078C0072CD0606801285C
:101420001BD0316802281CD0890734D5716889081F
:10143000890001437160FFF78DFE7168074662689D
:101440000C2001409200914215D0FFF783FEC11B92
:101450002048814208D90320F8BD316889031AD594
:10146000E4E7890117D5E1E770680C21084061685D
:1014700089008842E9D115480168C907C90FA94206
:101480000BD9016849084900294301600068C00779
:10149000C00FA84201D00120F8BD2078400706D532
:1014A0007068072109028843E1680843706000F012
:1014B00027F87168084A0906090F515CC8400749B6
:1014C00008600320FFF79EFE0020F8BD00200240C8
:1014D0000010024088130000B437000834000020D8
:1014E0000448054900684968044A4905490F515CA8
:1014F000C84070473400002000100240C437000884
:1015000010B514A00FC888B06C460FC415A00FC842
:101510000FC4184A53680C20194601401648042984
:1015200016D0082914D19902090F6C46645CD16A5F
:1015300004AA0907090F525CD90305D500231946EF
:10154000FEF7FAFD214601E020460C4901F0CEFEEF
:1015500008B010BD02030405060708090A0B0C0DAC
:101560000E0F10100102030405060708090A0B0CF0
:101570000D0E0F100010024000127A0000093D000D
:10158000002801D101207047F8B504460078EE4DDF
:10159000C00754D068680007800F012807D068682A
:1015A0000007800F022809D16868C00306D52868A3
:1015B000800344D56068002874D040E0606801284A
:1015C0000CD00121890400280DD0052825D02A68D7
:1015D000881082432A60286888430BE0286801212C
:1015E0000904084306E02868012212049043286099
:1015F0002868884328606068002812D0FFF7AAFD99
:101600000646286880031AD4FFF7A4FD801B6428CF
:1016100073D828688003F7D511E02868084328604C
:10162000DCE7FFF797FD06462868800307D5FFF73C
:1016300091FD801B642860D828688003F7D4207847
:10164000800741D568680007800F07D068680007E9
:10165000800F022809D16868C00306D42868800773
:1016600018D5E06801281DD114E0E068002828683A
:1016700019D0012108432860FFF76CFD0646286851
:10168000800707D4FFF766FD801B022835D828683D
:101690008007F7D52868F82188432169C9000843E5
:1016A000286011E04CE1400840002860FFF752FD3F
:1016B00006462868800707D5FFF74CFD801B0228E7
:1016C0001BD828688007F7D42078000727D5E06961
:1016D0000028686A12D0012108436862FFF73AFDCA
:1016E0000646686A80071AD4FFF734FD801B02287B
:1016F00003D8686A8007F7D511E08BE04008400006
:101700006862FFF727FD0646686A800707D5FFF77E
:1017100021FD801B02287DD8686A8007F7D42078D5
:1017200004264007002866DAE8690027C00007D4CD
:10173000E869B1060843E861E869084001270090BC
:1017400082480168C90515D40168801501437F48A6
:101750000160FFF7FFFC00907C480068C00509D4D9
:10176000FFF7F8FC0099401A64287DD87748006894
:10177000C005F5D5A06801280AD0002801D00528A9
:101780001ED0286A400840002862286AB04302E060
:10179000286A012108432862A068002814D0FFF7B6
:1017A000D9FC0090286A80071ED4FFF7D3FC00996B
:1017B000411A6748814257D8286A8007F5D513E057
:1017C000286A30432862E3E7FFF7C4FC0090286AE8
:1017D000800709D5FFF7BEFC0099411A5C48814299
:1017E00042D8286A8007F5D4002F04D0E869012187
:1017F00009078843E8612078C0061BD56069012885
:1018000034D0401D686B4ED030436863686B40082D
:10181000400000E028E06863FFF79CFC0646686B28
:10182000800707D5FFF796FC801B02281CD8686B41
:101830008007F7D4206A002868D069680907890FF3
:10184000022968D001263606022828682ED0B04327
:101850002860FFF77FFC04462868800172D5FFF7F7
:1018600079FC001B022852D90320F8BD686B304375
:101870006863686B012108436863FFF76BFC0646E9
:10188000686B800707D4FFF765FC801B0228EBD844
:10189000686B8007F7D5686BF8218843A169C90098
:1018A00008436863C6E7B0436863F4E7B043286061
:1018B000FFF750FC07462868800107D5FFF74AFC70
:1018C000C01B0228D0D828688001F7D4E86AE16AF2
:1018D000000900010843E862616AA06A0843696878
:1018E0003D22120491430843686028683043286011
:1018F000FFF730FC04462868800123D4FFF72AFC58
:10190000001B0228B0D828688001F7D51AE02868A3
:101910008001A4D416E00128A7D06868E96A0122F2
:101920001204636A02409A420AD10907E26A090F67
:10193000914205D10F2189040840A16A884201D053
:101940000120F8BD0020F8BD0010024000700040EA
:10195000881300000B4910B4401E884202D910BC05
:10196000012070470849486108480722C3691B02E3
:101970001B0A4C042343C361002088610A6110BC28
:1019800070470000FFFFFF0000E000E004ED00E012
:1019900070477047002801D10120704770B5054697
:1019A00004462035687F002803D12877204600F0C0
:1019B00015F802206877211D206801F057F80120F2
:1019C0004034A071A877E87720706070A070E07054
:1019D000207160716877002070BD000008B5006854
:1019E000094988420FD10948C26981150A43C26179
:1019F000C06900220840009001211320FFF744FC39
:101A00001320FFF735FC08BD002000400010024005
:101A1000014620314A7F012A01D00120704702226D
:101A20004A770168CB6801221343CB6000680849FC
:101A3000884202D00749884204D181684907490F8A
:101A4000062902D0016811430160002070470000A0
:101A5000002C014000040040704770B50446006847
:101A600001690025C9438907002915DBC168C943FD
:101A7000890711D4E91E016101202077206880695F
:101A80008007204602D0FFF7E7FF04E000F096F859
:101A9000204600F04FF9257720680169C9434907BE
:101AA00017D4C168C943490713D40421C94301614C
:101AB00002202077206880698005800F204602D0B0
:101AC000FFF7CAFF04E000F079F8204600F032F991
:101AD000257720680169C943090716D4C168C9433D
:101AE000090712D40821C943016104202077206826
:101AF000C0698007204602D0FFF7AEFF04E000F087
:101B00005DF8204600F016F9257720680169C94381
:101B1000C90617D4C168C943C90613D41021C943E3
:101B20000161082020772068C0698005800F204669
:101B300002D0FFF791FF04E000F040F8204600F0EB
:101B4000F9F8257720680169C943C90708D1C16838
:101B5000C943C90704D1891E0161204600F05EF91E
:101B600020680169C943090609D4C168C943090647
:101B700005D48021C94301612046FFF709FF206891
:101B80000169C943490609D4C168C943490605D456
:101B90004021C9430161204600F041F920680169F4
:101BA000C943890609D4C168C943890605D42021DF
:101BB000C94301612046FFF7ECFE70BD704700008D
:101BC000F8B504460020264620360090307F0D46AA
:101BD00001280FD0012004273077002A0CD0042AD6
:101BE0001CD0082A2FD00C2A3FD00090002030773C
:101BF0000098F8BD0220F8BD206800F083FF20683F
:101C0000816908221143816120688169B94381613A
:101C1000206881692A6911438161E7E7206800F043
:101C2000AFFF206881690122D202114381612068DF
:101C30008169521091438161206881692A69120289
:101C400011438161D2E7206800F0D6FF2068C169A6
:101C500008221143C1612068C169B943C16120688C
:101C6000C1692A691143C161C0E72068016A012284
:101C7000120391430162026A4168C76973231B0220
:101C80009F432B681B023B4301277F03BA43AF6886
:101C90003F031743124A904205D0124A904202D0A5
:101CA000114A904205D10122920391436A6992013F
:101CB00011434160C3616968016407622068C169BA
:101CC0000122D2021143C1612068C16952109143BF
:101CD000C1612068C1692A6912021143C16185E7A7
:101CE000002C01400044014000480140002801D17F
:101CF0000120704770B5054604462035687F0028EE
:101D000003D12877204600F014F802206877211DBF
:101D1000206800F0ABFE01204034A071A877E8777E
:101D200020706070A070E070207160716877002092
:101D300070BD70477047000030B50246044600256C
:101D400020324030002908D0042908D0082908D0C2
:101D50004378012B07D0012030BD937FF9E7D37F73
:101D6000F7E70378F5E7022300290ED004290ED007
:101D700008290ED0437000290DD0042910D008295D
:101D800014D00C2918D001253DE09377F3E7D377E1
:101D9000F1E70370EFE72068C2681A43C26010E001
:101DA0002068C26804231A43C2600AE02068C2683F
:101DB00008231A43C26004E02068C26810231A4353
:101DC000C2600122206800F08FFE104A2068904215
:101DD00005D00F49884202D00E49884204D1416C97
:101DE0000123DB031943416420680123904202D0A0
:101DF0000949884204D181684907490F062902D060
:101E0000016819430160284630BD0000002C0140E4
:101E10000044014000480140000400407047704702
:101E20007047F8B5816F0446C66F00688268254622
:101E3000120610278035002A26DA212924D1EFF353
:101E40001081012282F31088826880239A43826085
:101E500081F31088E06E002808D0FEF761FE0028AC
:101E600004D0E06EFEF7A1FE20282FD0EFF3108102
:101E7000012080F3108820680268C0239A43026022
:101E800081F310882020A0672068816849061BD54F
:101E9000222E19D1EFF31081012282F3108882687B
:101EA00040239A43826081F31088206F002808D075
:101EB000FEF736FE002804D0206FFEF776FE2028BD
:101EC00004D0204601F02AF80020F8BD2F6003203E
:101ED000F8BD7047F8B502680446D0691168966885
:101EE0009F4B05461D402023002D76D0F7079D4DC2
:101EF000FF0FBC460D402F436ED02546C7078035E7
:101F0000002F06D0CF0504D5012717622A683A436F
:101F10002A60820708D5F20706D0276802223A62B3
:101F20002A6804273A432A60420708D5F20706D0F8
:101F30002668042232622A68022632432A60020797
:101F40000AD50A461A406646324305D0266808225A
:101F500032622E6816432E60020508D54A0106D566
:101F600001222668D20232622A681A432A602A684D
:101F7000002A2FD0800606D5880604D5616E002978
:101F800001D020468847286821688968490602D41C
:101F9000282108422DD0204600F0C0FF206881682B
:101FA000490622D5EFF31081012282F3108883685D
:101FB00040229343836081F31088206F002814D05F
:101FC00069494163206FFEF7CCFD002802D0206FE5
:101FD000416B8847F8BD00E011E085060FD58D06FE
:101FE0000DD5616E00297CD1F8BD2046FFF771FF49
:101FF000F8BD2046FFF76DFF00202860F8BD256E74
:10200000012D6FD1C5066DD5CD066BD51027176292
:1020100020688168254649064035002948DA226F44
:10202000116849680904090CE8D02E8B8E42E5D965
:1020300069839169202933D0EFF31081012282F363
:10204000108802683E01B243026081F31088EFF30A
:102050001081012080F310882068826852085200A5
:10206000826081F31088EFF31081012080F31088E3
:102070002068866840229643866081F31088E36773
:1020800000202066EFF31081012080F31088206883
:102090000368BB43036081F31088206FFEF740FDA7
:1020A000288B698B401A81B22046FFF7B9FEF8BD34
:1020B000298B6A8B891A6A8B89B2002AF7D000298A
:1020C000F5D0EFF31082012585F310880568FF260F
:1020D0002136B543056082F31088EFF310820120AA
:1020E00001E023E01BE080F31088206885686D081C
:1020F0006D00856082F31088E36700202066EFF3AF
:1021000010826066012080F3108820680368BB435A
:10211000036082F310882046FFF782FEF8BD0506B3
:1021200007D50D0605D5A16E0029F7D020468847B2
:10213000F8BD4006FCD54806FAD52046EFF31081DD
:10214000012484F3108814684025AC43146081F3A3
:10215000108883670021816600F050F9F8BD000007
:102160000F08000020010004A52D0008002801D15F
:102170000120704710B50446806F002805D100216A
:1021800074200155204600F027F82420A06720681D
:102190000168490849000160204600F0EFFE01286F
:1021A00018D0606A002802D0204600F063FD206845
:1021B00041680122D202914341602068816808226F
:1021C000914381602068016801221143016020462B
:1021D00000F0B6FD10BD0000F0B587B00024054644
:1021E0000094019402940394049400683149884255
:1021F0005DD131488269012189030A438261826984
:102200000A4005924269C9000A4342614069084098
:1022100005900320400200900220019003200390CB
:102220000120049009206946C006FEF7D1FE244E25
:1022300080277460B46034617461F7601F48B461D2
:1022400030608014F0613046FEF706FD002801D0B2
:10225000FEF794F92E6775621B4E1A483060B46021
:1022600034617461F7601020B46170600002F06145
:102270003046FEF7F1FC002801D0FEF77FF9134845
:102280000168421511430160EE66002211461B20D1
:102290007562FEF7F9FF1B20FEF7EAFF0C4B18688A
:1022A000026810210A43026019685020086207B0D2
:1022B000F0BD000000380140001002403000024034
:1022C0001C04002044000240600400200000014083
:1022D0009803002070B5C36F202B2BD100290BD0A1
:1022E000002A09D0012483682403A34206D103698C
:1022F000002B03D1CB0701D0012070BD0346603312
:102300001C7D012C16D001241C7500230366036874
:102310005C6824020BD5EFF31084012585F3108847
:102320001D680126B60635431D6084F3108800F051
:10233000B5FE70BD022070BD70477047F8B5044609
:10234000806F202852D100290BD0002A09D0012308
:10235000A0681B03984206D12069002803D1C80752
:1023600001D00120F8BD25466035287D01283DD0EB
:102370000120287520464030E16402824282002715
:102380002646803637602120A067E06E00281BD0EB
:1023900017498162E16E1748C862E16E164808630A
:1023A000E06E134647632068E16C2830844662463D
:1023B000E06EFEF785FC002806D0102030602F75F7
:1023C0002020A0670120F8BD2168402008622F75F9
:1023D000EFF31081012080F3108820688268802349
:1023E0001A43826081F310880020F8BD0220F8BDF6
:1023F000C92E0008132F0008B92D00087047704738
:10240000FEE70000F0B55A4C87B0A01CFEF772F84A
:102410000590201DFEF76EF8074606212046FEF7C0
:102420006FF8060AC5B20598012802D0FF2831D0FE
:1024300058E0022F7AD14E4A9079B04276D1D079C5
:10244000A84273D14B4BD95701290CD10C20185EEF
:10245000494D0446FF342C34AC4204D8002800DA3D
:10246000404240429881454C10782070507860700E
:102470000420A07098890212E27020710812607125
:10248000A17107212046FEF73BF8010AE171207295
:10249000092049E0012F49D135488179B14245D120
:1024A000C079A84242D136A01EC80394029301927B
:1024B00000910068049000246846FDF7A2FE002801
:1024C0000AD96846015D2D480155641CE4B268468E
:1024D000FDF797FEA042F4D86846FDF792FEC0B221
:1024E00001F00EF805980221022821D003281DD101
:1024F000012F1BD11E488279B24217D1C279AA425C
:1025000014D11E4C02782270407860701948A17076
:10251000C08A0112E170207105212046FDF7F0FF0D
:10252000010A6171A071072000F0EAFF07B0F0BD59
:10253000012FFBD10E488279B242F7D1C279AA426B
:10254000F4D10E4C02782270407860700948A17076
:10255000808A010AE170207105212046FDF7D0FF35
:10256000010A6171A071072000F0CAFF07B0F0BD39
:102570004C02002000000020560200002C02002027
:102580004443452D323330322D56342E315F48418D
:102590004C000000F8B5454EB188B01C49BA0CB2E9
:1025A000FDF7A8FF054606213046FDF7A9FF0146C5
:1025B0003F4F0020325C3A54401CC0B20628F9D389
:1025C0000A0ABA71C9B23B48F9710F2D04D0022D25
:1025D0002AD0032D3FD064E0B3799A4261D1F279D9
:1025E00091425ED1611EF6290DD84481012080F30D
:1025F000108800F0A7FF002853D180F310883078AE
:1026000000280DD14DE0FF20387178710621274850
:10261000FDF776FF010AB971F8713078002840D0D3
:10262000082000F06DFF3CE0B3799A4239D1F2798D
:10263000914236D1204A611E914232D8A1B28182A4
:102640001E4800684163012080F3108800F07AFF83
:10265000002820D025E0B3799A4222D1F279914224
:102660001FD11749174A611891421AD822460A21E8
:102670004A430C210546415E1046FDF749FDE882BC
:10268000012C01D10A20E882012080F3108800F09B
:1026900059FF002805D1002080F31088082000F0A1
:1026A0002FFF20210148FDF7A1FDF8BD4C020020BD
:1026B0002C02002000000020E7030000500300204F
:1026C000E40C0000C819000010B584B000211848BF
:1026D00000910191154A0291026081600124520526
:1026E00004614260C16004224261017641768476D1
:1026F000FF22C176C232C2610E4A01621171846248
:10270000FEF770F8002801D0FDF738FF0120000324
:10271000019007200290009469460548FDF76EFF7E
:10272000002801D0FDF72AFF04B010BD00240140AD
:10273000BC020020DC02002008B5104841690122DB
:10274000114341614069012110400090002209209D
:10275000FEF79AFD0920FEF78BFD002201210A20D9
:10276000FEF792FD0A20FEF783FD002201210B20D7
:10277000FEF78AFD0B20FEF77BFD08BD001002402E
:1027800030B587B00024304800940194029403943B
:1027900004944269012189050A43426142690A4061
:1027A0000592426949110A43426142690A40059211
:1027B000426949000A434261406909250840ED0623
:1027C0000590012210212846FEF7BDFC00222021A1
:1027D0002846FEF7B8FC0820009031200004019044
:1027E000694602942846FEF7F3FB0121302001914F
:1027F00003910090029469462846FEF7E9FB4020C9
:1028000000900194694602942846FEF7E1FB80207F
:102810000090112000040190694602942846FEF7BA
:10282000D7FB002202210620FEF72EFD0620FEF730
:102830001FFD002211460720FEF726FD0720FEF7A8
:1028400017FD07B030BD00000010024010B5094868
:1028500007490160062141600749C160272109013C
:102860008160FEF77DFC002801D0FDF787FE10BDDA
:102870000030004040030020FF0F000070B58EB014
:10288000002400940194244D02940394049405942C
:10289000204E06942E600120AC6068602C611F48B9
:1028A000AC61E8602846FFF775F8002801D0FDF715
:1028B00065FE1948FFF71AFA002801D0FDF75EFE01
:1028C00060200090FF202D30019002940022694684
:1028D00004941148FFF774F9002801D0FDF74EFE6B
:1028E0000794089409940A940B942868B0420FD175
:1028F0000B484269012189040A434261406908404A
:102900000C9002200790089007A90648FEF760FB8C
:102910000EB070BD0020004050030020E70300000F
:10292000001002400004004810B50C480A4901603C
:102930004B21C901416000218160C1600161816159
:10294000C1610C22016242614162FFF70FFC002865
:1029500001D0FDF713FE10BD0038014098030020A0
:10296000FEE77047704700B500F002F800BD0000B8
:1029700030B4194B58680124002804D05868401E10
:10298000586000D11C70154D00210C20484340199F
:102990004268002A09D04268521E426005D1447044
:1029A0000278012A01D182684260491CC9B2042917
:1029B000EBD39868401C98609868094A00219042BF
:1029C00000D199605878401CC0B258700A2800D3D2
:1029D000597030BC704700001C0000208C020020A1
:1029E000FFFFFF7F70B594B00024059404940F940A
:1029F000092002250E9400901394E8030294039496
:102A0000069409900B940C940D94012600011094E7
:102A1000119412940A900196079608956846FEF75D
:102A2000AFFD002801D072B6FEE707200C900E948F
:102A300001210D950F940CA8FEF7C4FC002801D0CD
:102A400072B6FEE710A810961294FEF73FFC00281D
:102A500001D072B6FEE714B070BD704710B50248E1
:102A6000FEF7FBFF10BD00005003002070B40268A9
:102A7000184C194EA04201D0B04204D11346702523
:102A80004A68AB431A43154B154DA04208D0B042DB
:102A900006D0144EB04203D0984201D0A84204D1CF
:102AA00003263602B243CE6832438026B2434E69D3
:102AB000324302608A68C2620A688262A04203D01E
:102AC000984201D0A84201D1096901630121416105
:102AD00070BC7047002C01400004004000440140DD
:102AE000004801400020004010B4C906C90E01236F
:102AF000046A8B409C430462036A8A401343036266
:102B000010BC7047F0B4026A520852000262056AB3
:102B1000436882697024A24392080C6892001443AF
:102B2000022295438A68134E2A43134FB04204D0C1
:102B3000B84202D0114DA84206D10825AA43CD685B
:102B40001543042295432A46B04204D0B84202D02D
:102B50000A4DA84206D103252D02AB434D691D4302
:102B60008B692B4343608461496841630262F0BC16
:102B700070470000002C0140004401400048014023
:102B8000F0B4026A10239A430262046A43688269BD
:102B900073252D02AA430D68144E2D0215432022E1
:102BA00094438A6812012243B04207D11446CA688E
:102BB0008027BC43120122434024A243B04205D0E7
:102BC0000B4CA04202D00B4CA04208D10324A4021B
:102BD000A3434C69A4001C438B699B0023434360BF
:102BE0008561496881630262F0BC7047002C014036
:102BF0000044014000480140F0B4026AFF23013361
:102C00009A430262046A4368C2697025AA43920823
:102C10000D68920015430122520294438A68124EB5
:102C200012022243B04207D11446CA68C714BC43FB
:102C3000120222430415A243B04205D00B4CA0421D
:102C400002D00B4CA04208D103242403A3434C69B7
:102C500024011C438B691B0123434360C561496800
:102C6000C1630262F0BC7047002C01400044014087
:102C70000048014010B4818CC90707D001684A6838
:102C800001235B049A43836A1A434A60818C890753
:102C900007D501684A6801231B049A43C36A1A4393
:102CA0004A60818C490707D501684A6801239B0463
:102CB0009A43036B1A434A60818C090707D5016860
:102CC0004A680123DB039A43436B1A434A60818CB1
:102CD000C90607D501688A6801231B039A43836BE1
:102CE0001A438A60818C890607D501688A680123A6
:102CF0005B039A43C36B1A438A60818C490612D5E1
:102D000001684B6801221205046C934323434B6016
:102D1000016C914207D101684A6803235B059A431D
:102D2000436C1A434A60818C090607D501684A68DA
:102D30000123DB04806C9A4302434A6010BC704755
:102D4000F8B50446002580300560FEF703FA074613
:102D500020680068124E000709D501213B46002279
:102D600049052046009600F0F3F900280DD12068AF
:102D7000006840070BD501213B460022890520460B
:102D8000009600F0E5F9002801D00320F8BD2020CE
:102D9000A067E0672566603425750020F8BD000057
:102DA000FFFFFF0110B5406A0022014640314A830F
:102DB0004A82FFF78EF810BD70B5446AA06FE26FCB
:102DC0002168896800230906002911DA21280FD11A
:102DD00052200353EFF31081012080F31088206804
:102DE0000568C026B543056081F310882020A067E0
:102DF00020688068400606D5222A04D15A20035351
:102E0000204600F08BF820468030016810221143E4
:102E100001602046FFF75DF870BD10B50146896975
:102E2000406A202937D000225A210A52EFF310823B
:102E3000012181F3108801680B68FF240134A3434A
:102E40000B6082F31088EFF31082012181F3108868
:102E500001688B685B085B008B6082F31088EFF37E
:102E60001082012181F3108801688B684024A343FC
:102E70008B6082F310882021C167016E01290AD17D
:102E8000EFF3108281F3108801680B681024A343CC
:102E90000B6082F31088016E012902D0FFF74CFA13
:102EA00010BD5821095AFEF7BBFF10BD10B5406A8E
:102EB000016E012902D0FFF740FA10BD5821095ACE
:102EC0004908FEF7ADFF10BD10B501468969406A9B
:102ED00020291BD0002252210A52EFF31082012137
:102EE00081F3108801688B688024A3438B6082F390
:102EF0001088EFF31081012282F3108800680268C5
:102F000040231A43026081F3108810BDFFF776FA60
:102F100010BD10B5406AFFF772FA10BD10B4EFF3A0
:102F20001082012181F3108801680B68FF2421348D
:102F3000A3430B6082F31088EFF31082012181F329
:102F4000108801688B685B085B008B6082F31088D7
:102F5000016E01290AD1EFF3108281F31088016814
:102F60000B681024A3430B6082F310882021C167F3
:102F700000210166416610BC7047000070B5044630
:102F800081680069E26901436069002510430143DB
:102F9000206802683C4B1A400A430260206841687E
:102FA000032212039143E26811434160216AA06940
:102FB0000143206882680B231B029A430A43826004
:102FC0003248006B8007800F06D0012816D00228F7
:102FD00016D0032810D010200122E369D2032C4917
:102FE0002C4E93422AD100280CD002280DD0042860
:102FF0000DD008283ED10EE00220EDE70420EBE7DB
:103000000820E9E7FEF76CFA03E00A4603E0FEF762
:1030100077FA020032D0616850004A088018FDF744
:1030200061F880B201461039B14223D81A490140F3
:103030000007420F20680A43C2601FE0002806D044
:10304000022807D0042807D0082813D108E0FEF78B
:1030500047FA03E00A4603E0FEF752FA02000DD0F9
:10306000616848088018FDF73DF880B201461039C4
:10307000B14201D9012501E02168C86000206066E5
:10308000A066284670BD0000F369FFFF00100240F3
:1030900000127A00EFFF0000F0FF0000F8B50446D0
:1030A0004165403000272646028380363760222063
:1030B000E0672546206F603500281BD021498162DA
:1030C000216F2148C862216F20480863206F134692
:1030D0004763606D2168844662462431206FFDF7A6
:1030E000EFFD002806D0102030602F752020E0670B
:1030F0000120F8BD2F75EFF31081012080F31088B7
:1031000020680268FF2301331A43026081F31088AC
:10311000EFF31081012080F310882068836801227A
:103120001343836081F31088EFF3108182F31088DA
:103130002068826840231A43826081F3108800204F
:10314000F8BD00001B2E0008AD2E0008B92D0008A8
:10315000FFB50446006881B00E460A9DC169174656
:10316000304688433FD00020B84268D120466030C6
:103170000090681C5BD0FDF7EDFF0499401AA8424F
:1031800033D8002D31D02068016849074FD5C06978
:10319000C04300054BD401202168C0020862EFF350
:1031A0001081012080F3108820680268FF23A1337A
:1031B0009A43026081F31088EFF31081012080F3BD
:1031C00010882068826852085200826081F310885B
:1031D0002020A067E06780342060009900200875F7
:1031E000032005B0F0BD0120BEE7EFF31081012000
:1031F00080F3108820680268FF23A1339A4302609D
:1032000081F31088EFF31081012080F3108820688B
:10321000826852085200826081F310882020A067E3
:10322000E067009900200875032005B0F0BD206814
:10323000C1693046884305D00020B84299D00020AB
:1032400005B0F0BD0120F8E710B51148FEF742FEC9
:103250000F480068C169C943C90618D4102101622A
:103260000C4C2078002812D10948FEF7DAFD0A48F4
:10327000006840682021081AC2B222700749084835
:10328000FCF79BFF202205490148FFF723F810BDFA
:1032900098030020000000201C0400206C02002085
:1032A0004C02002010B50F480F4C0278417863891A
:1032B000204600789A4201D1082802D0002A08D07E
:1032C0000DE0032902D0062909D106E0FFF79AF89C
:1032D00005E0082803D1062901D1FFF75BF900209A
:1032E000207010BD4C02002000000020F0B4040C3F
:1032F0008BB2264682B25E430D0C1046370C584303
:10330000360480190021794116466E43370C360485
:103310008019794126466E438919F0BC704702E056
:1033200008C8121F08C1002AFAD170477047002050
:1033300001E001C1121F002AFBD17047042806D208
:103340000C214843054940184178012901D000204B
:103350007047002141700120704700008C0200205E
:10336000042800D3FEE7012282F310880C22064BCA
:103370005043C218516091600021517001221A54CB
:1033800081F31088704700008C02002000280ED0C6
:10339000012800D10220012181F3108804494860EE
:1033A0000020087080F3108808780128FCD170474D
:1033B0001C000020FDF716FFFFF714FBFFF7E0F9F4
:1033C000FFF7BAF9FFF780F9FFF7AEFAFFF73EFA19
:1033D000FFF754FA3C493D4A08883D4B10800028CD
:1033E00001D0984201D1012010804888394A002834
:1033F000108001D0984202D17D20C0001080364A52
:1034000080B2126850630420085E344900280880A6
:1034100001D0401C01D10A2008803148FDF7DAFEB6
:103420002D48FEF7F5FA00212B48FEF785FC2D48C4
:10343000FEF7F7FC20222C492A48FEF74BFFFA2220
:103440002A492B48FDF7DCFA092000222021C0067A
:10345000FDF779FE32210020FFF782FFFF21F531D1
:103460000120FFF77DFF23490220FFF779FF0225A6
:10347000214E224C00270020FFF760FF002809D0D2
:103480001B48FDF70FFBFCF7EBFFFA221749184822
:10349000FDF7B6FA0120FFF751FF002807D01048CA
:1034A000FDF798FE09201021C006FDF744FE02201A
:1034B000FFF744FF002800D0357020780028DAD0CC
:1034C000FFF7F0FE2770D6E7003C00080A00002056
:1034D000FFFF000014000020500300201600002011
:1034E00040030020980300206C02002038000020D8
:1034F000BC02002088130000020000200000002011
:1035000070B509240546E406012220212046FDF776
:103510001AFE2A4608490948FEF710FF0848FDF739
:1035200046FB0128FAD10520FFF730FF00222021B9
:103530002046FDF708FE70BD2C02002098030020F5
:103540006004002010B586B0002000900190029029
:10355000164C012003940490FDF7AEFC05A902A8C7
:10356000FDF7F4FB002802D0012006B010BD104A80
:10357000694650890870000A4870908A8870000A6D
:10358000C870D08A08710012487121460320019B3F
:10359000009AFDF74DFC002802D0032006B010BDB4
:1035A000FDF73CFC002006B010BD0000003C000808
:1035B0000000002000C1814001C0804101C0804165
:1035C00000C1814001C0804100C1814000C18140F3
:1035D00001C0804101C0804100C1814000C18140E3
:1035E00001C0804100C1814001C0804101C08041D3
:1035F00000C1814001C0804100C1814000C18140C3
:1036000001C0804100C1814001C0804101C08041B2
:1036100000C1814000C1814001C0804101C08041A2
:1036200000C1814001C0804100C1814000C1814092
:1036300001C0804101C0804100C1814000C1814082
:1036400001C0804100C1814001C0804101C0804172
:1036500000C1814000C1814001C0804101C0804162
:1036600000C1814001C0804100C1814000C1814052
:1036700001C0804100C1814001C0804101C0804142
:1036800000C1814001C0804100C1814000C1814032
:1036900001C0804101C0804100C1814000C1814022
:1036A00001C0804100C1814001C0804101C0804112
:1036B00000C1814000C0C101C30302C2C60607C7E2
:1036C00005C5C404CC0C0DCD0FCFCE0E0ACACB0B52
:1036D000C90908C8D81819D91BDBDA1A1EDEDF1F82
:1036E000DD1D1CDC14D4D515D71716D6D21213D372
:1036F00011D1D010F03031F133F3F23236F6F73722
:10370000F53534F43CFCFD3DFF3F3EFEFA3A3BFB11
:1037100039F9F83828E8E929EB2B2AEAEE2E2FEFC1
:103720002DEDEC2CE42425E527E7E62622E2E32331
:10373000E12120E0A06061A163A3A26266A6A76761
:10374000A56564A46CACAD6DAF6F6EAEAA6A6BABD1
:1037500069A9A86878B8B979BB7B7ABABE7E7FBF01
:103760007DBDBC7CB47475B577B7B67672B2B373F1
:10377000B17170B0509091519353529296565797A1
:10378000559594549C5C5D9D5F9F9E5E5A9A9B5B91
:1037900099595898884849894B8B8A4A4E8E8F4F41
:1037A0008D4D4C8C448485458747468682424383B1
:1037B000418180400000000000000000010203047D
:1037C000060708090000000001020304EC370008A6
:1037D00000000020380000001E33000824380008D4
:1037E00038000020900800002E330008000101007E
:1037F00000000000000000000000000000000000C9
:103800000000000046000000000000000000000072
:1038100000000000010000000400000000000000A3
:0438200000127A0018
:04000005080000B13E
:00000001FF
